:10000000F2C000000BC1000009C1000007C10000E0
:1000100005C1000003C1000001C10000FFC00000D5
:10002000FDC00000FBC00000F6C1000034C20000AB
:10003000F5C00000F3C00000F1C00000EFC00000F8
:10004000EDC00000EBC00000E9C00000E7C0000008
:10005000E5C00000E3C00000E1C00000DFC0000018
:10006000DDC00000DBC00000D9C00000D7C0000028
:10007000D5C00000D3C00000D1C00000CFC0000038
:10008000CDC00000CBC00000C9C00000C7C0000048
:10009000C5C00000C3C00000C1C00000BFC0000058
:1000A000BDC00000BBC00000B9C000004284A483F2
:1000B0000124C3040274A344C282E364D4430381D1
:1000C00023146394B4C40A000A00206469740020F5
:1000D000646168004368617220000A004F707073A9
:1000E0002C20756E737570706F7274656420636810
:1000F000617261637465723A200053706163650ACE
:1001000000444F455320414E59424F4459205354C7
:10011000494C4C204B4E4F57204D4F525345204396
:100120004F44453F00534F5300000100006001124F
:10013000000200007201220022000094011500213B
:10014000000084010900030000A90104010309045F
:10015000AD011402030904C30120000001C12600FF
:100160001201000200000020C01679040001010203
:10017000000109022200010100C03209040000014F
:100180000300000009211101000122150007058369
:10019000032000010631FF0974A1537508150026DC
:1001A000FF00952009758102C00403090414035956
:1001B000006F007500720020004E0061006D006548
:1001C000000000200359006F0075007200200055E8
:1001D000005300420020004400650076006900637F
:1001E00000650000000011241FBECFEFDAE0DEBF83
:1001F000CDBF11E0A0E0B1E0E8E7F7E002C0059074
:100200000D92A030B107D9F711E0A0E0B1E001C034
:100210001D92A330B107E1F779D0ACC2F1CE0F93B4
:100220001F93CF93DF93182F803269F48AEF90E009
:100230008DD280EE95E120E931E0F9013197F1F7B7
:100240000197D9F74EC081548A3148F08CED90E087
:100250007DD2812F9AD08AED90E078D242C084ED91
:1002600090E074D2812F91D08AE38FD0E12FF0E01B
:10027000E559FF4FE4910E2F07701E2FC0E9D1E022
:1002800022C05E9A17FF0BC08FEC90E05FD280E631
:1002900099E0FE013197F1F70197D9F70AC08AEC8E
:1002A00090E054D280E293E0FE013197F1F701979C
:1002B000D9F75E9880E293E0FE013197F1F701975C
:1002C000D9F7110F01500023E1F688EC90E03ED2FF
:1002D00080E496E020E931E0F9013197F1F70197E8
:1002E000D9F7DF91CF911F910F910895CF93DF93AD
:1002F000EC01FE0121968491882311F090DFF9CF63
:1003000086EC90E023D2DF91CF9108951F93CF9395
:10031000DF9380E88093610010926100569A5E98A6
:100320001DD010E0C0E9D1E00BC085E291E0DEDF36
:1003300088E99AE3FE013197F1F70197D9F71F5F3A
:10034000163098F381E091E0D1DF80E49CE9FE0172
:100350003197F1F70197D9F710E0E7CF81E080936B
:10036000D70080EA8093D80082E189BD09B400FEFD
:10037000FDCF80E98093D8001092E0001092000138
:100380008CE08093E20078940895482F80910001DA
:10039000882309F43EC02FB7F89483E08093E900E6
:1003A00080910201882341F08091E80085FD02C020
:1003B0002FBF12C0109202019091E4009C5F33E0C5
:1003C0008091E80085FD13C02FBF8091E40089175C
:1003D00029F481E0809302018FEF0895809100015C
:1003E0008823B9F02FB7F8943093E900E9CF409310
:1003F000F1008091E80085FD06C08AE38093E80063
:100400001092010103C082E0809301012FBF80E0C0
:1004100008958FEF08951F920F920FB60F92112437
:100420008F939F938091E1001092E100982F83FFBA
:100430000FC01092E90081E08093EB001092EC0075
:1004400082E28093ED0088E08093F000109200013A
:1004500092FF1AC0809100018823B1F080910101C0
:10046000882391F0815080930101882369F483E00F
:100470008093E90002C01092F1008091E80085FDB0
:10048000FACF8AE38093E8009F918F910F900FBE7F
:100490000F901F9018951F920F920FB60F92112474
:1004A0002F933F934F935F936F937F938F939F937C
:1004B000AF93BF93CF93DF93EF93FF931092E90035
:1004C0008091E80083FF2CC14091F1003091F10050
:1004D0008091F100A82FB0E02091F100922F80E0F0
:1004E000A82BB92B8091F100682F70E02091F100CA
:1004F000922F80E0682B792B8091F100C82FD0E0FB
:100500002091F100922F80E0C82BD92B82EF8093AD
:10051000E800363009F056C020E331E0A90145502B
:100520005040F9013797859194918A179B07E1F420
:10053000FA018591949186179707B1F49A012E5F7D
:100540003F4FF901659174912E5F3F4FF90124915E
:10055000CE01CF3FD10519F010F08FEF90E0422F80
:10056000821758F4482F09C0295F3F4F495F5F4FFA
:10057000F1E021363F07A9F6D3C05EEF8091E80095
:10058000282F30E0C90185709070892BB9F322FDC6
:10059000CAC0342F413208F030E2232FCB0106C00D
:1005A000FC010196E491E093F10021502223C1F770
:1005B000630F711D431B5093E8004423F9F630325A
:1005C000E9F2B1C0353061F48EEF8093E80080919C
:1005D000E80080FFFCCF8A2F80688093E300A3C0EF
:1005E000393031F5442309F09BC0A09300018EEF10
:1005F0008093E8008AE591E021E02093E900FC0186
:100600000196E491E093EB00EE2369F0AC014F5FBB
:100610005F4FFC0184918093EC00CA010196FA01BE
:1006200034913093ED002F5F253039F78EE14DC0C6
:10063000383061F4403809F073C08091E80080FFE1
:10064000FCCF809100018093F1001BC03323E9F4BB
:100650008091E80080FFFCCF423811F080E00DC0AF
:100660006093E9008091EB0090E025E096958795F6
:100670002A95E1F781701092E9008093F1001092C1
:10068000F1008EEF8093E8004EC0313019F0333026
:1006900009F046C04230F1F4AB2BE1F4262F2F775E
:1006A000822F81508430B0F48EEF8093E800209345
:1006B000E9003330A9F189E18093EB0081E090E01B
:1006C00002C0880F991F2A95E2F78093EA001092E2
:1006D000EA0029C0313021F5413A11F5672B01F5C7
:1006E0004C2F5EEF8091E800282F30E0C901857023
:1006F0009070892BB9F322FD16C0942F413208F077
:1007000090E2892F03C01092F10081508823D9F71D
:10071000491B5093E800442329F7903219F303C092
:1007200081E28093EB00FF91EF91DF91CF91BF9138
:10073000AF919F918F917F916F915F914F913F9179
:100740002F910F900FBE0F901F9018951F93CF936E
:10075000DF93EC01FE0121961491112339F01A3038
:1007600011F48DE012DE812F10DEF4CFDF91CF91F6
:080770001F910895F894FFCFDA
:00000001FF
